S00F000053414D335334422E7372656338
S21440000070240020410140003F0140003F01400075
S2144000103F0140003F0140003F014000000000001B
S2144000200000000000000000000000003F0140000B
S2144000303F014000000000003F0140003F014000FB
S2144000403F0140003F0140003F0140003F0140006B
S2144000503F0140003F0140003F0140003F0140005B
S2144000603F0140003F0140003F0140003F0140004B
S2144000703F0140003F0140003F0140003F0140003B
S2144000803F0140003F0140003F0140003F0140002B
S2144000903F0140003F0140003F0140003F0140001B
S2144000A03F0140003F0140003F0140003F0140000B
S2144000B03F0140003F0140003F0140003F014000FB
S2144000C03F0140003F0140003F0140003F014000EB
S2144000D010B5054C237833B9044B13B10448AFF33D
S2144000E000800123237010BD2C0400200000000077
S2144000F0800340000C4B43B10C4810B50C49AFF39D
S21440010000800C48036823B910BD0A48036833B919
S2144001107047094B002BF7D0BDE810401847064BF8
S214400120002BF5D0184700BF0000000080034000B9
S2144001303004002080034000000000007047FEE7C7
S21440014008B51C4B1C4A9A4210D01C4B194A9A427E
S2144001500CD2013B9B1A23F0030304331344164985
S21440016051F8040B42F8040B9A42F9D1144B154A45
S2144001709A420AD2013B9B1A23F0030304331344EA
S214400180002142F8041B9342FBD10F4B23F0604200
S21440019022F07F020D498A6003F16043B3F5404F79
S2144001A003D28B6843F000538B60094B9847094B4A
S2144001B09847FEE700000020800340002C04002003
S2144001C06C0400202C0400200000400000ED00E0FD
S2144001D0E9014000D901400008B5024B984700208D
S2144001E008BD00BF3D01400070B50F4E0F4D761B59
S2144001F0B61018BF002405D0013455F8043B984784
S214400200A642F9D10A4E0B4D00F0A8F8761BB61060
S21440021018BF002406D0013455F8043B9847A64240
S214400220F9D170BD70BD00BF680340006803400050
S2144002307003400068034000024B13B1024800F0D0
S21440024005B87047000000005902400000230146F0
S2144002501A46184600F01EB838B50A4C0A4D641BBC
S214400260A4100AD004F18043013B05EB8305013C12
S21440027055F804399847002CF9D1BDE8384000F0CD
S21440028077B800BF800340007C034000704700BF43
S214400290704700BF2DE9F8432C4D0646286898461F
S2144002A00F469146FFF7F2FF294B1C68D4F84831B9
S2144002B0002B3ED05A681F2A1CDC02F1010E76B194
S2144002C0012103EB8204C4F88890D3F8880191405A
S2144002D00843022EC3F88801C4F8088123D00232AE
S2144002E0C3F804E0286843F82270FFF7D1FF0020E7
S2144002F0BDE8F883174B0BB34FF4C870AFF30080DC
S2144003000346D8B10020D4F848114FF0010E58608B
S21440031019600246C4F84831C3F88801C3F88C0116
S214400320002EDCD0CCE7D3F88C010143C3F88C1107
S214400330D5E704F5A673C4F84831BBE72868FFF74D
S214400340A7FF4FF0FF30BDE8F88300BF2804002029
S214400350580340000000000000000020F8B500BF31
S214400360F8BC08BC9E46704739024000F500400085
S214400370F8B500BFF8BC08BC9E467047D1004000A8
S21440038000000000EC02002054030020BC030020C4
S2144003900000000000000000000000000000000018
S2144003A00000000000000000000000000000000008
S2144003B000000000000000000000000000000000F8
S2144003C000000000000000000000000000000000E8
S2144003D000000000000000000000000000000000D8
S2144003E000000000000000000000000000000000C8
S2144003F000000000000000000000000000000000B8
S21440040000000000000000000000000000000000A7
S2144004100000000000000000000000000000000097
S2144004200000000000000000010000000000000086
S2144004300E33CDAB34126DE6ECDE05000B0000004B
S2144004400000000000000000000000000000000067
S2144004500000000000000000000000000000000057
S2144004600000000000000000000000000000000047
S2144004700000000000000000000000000000000037
S2104007A00000000000000000480400209C
S80440014179
